:100000008316FA308500BF30860057308100831296
:1000100005119101940195019601970198011930FC
:100020008E001A308F00853099001A30840080309D
:100030008000840A50300402031D17286400051A4A
:100040001E2892010E08840000088C00EA2064003B
:10005000051A7B2806089000901A3028101E0928DF
:10006000901E3A28101E3A280B30110203183A2825
:100070000C309100811F41288101921F920A111EAC
:10008000910A111A6228921F27289401950196015E
:10009000970198011A300F02031927284F300F02D9
:1000A000031927280F0384000130000203192728B1
:1000B0000F0884008E004F300F02031D8F0A01309D
:1000C0008000E528901E6728101E712843289101A2
:1000D0004F300E02031D6F2819308E0022288E0A21
:1000E0002228910119300E02031D79284F308E000D
:1000F00022288E0322280F0884008E004F300F0222
:10010000031D8F0A06088D008D130D138D120D121D
:100110001830800008300D020319E428CD3080002B
:1001200004300D020319E4289D3080000C300D02CC
:100130000319E4281B30800002300D020319E42863
:10014000973080000A300D020319E428D730800070
:1001500006300D020319E4281E3080000E300D0217
:100160000319E428DF30800001300D020319E42870
:100170009F30800009300D020319E428DE30800032
:1001800005300D020319E4285B3080000D300D02AC
:100190000319E428D130800003300D020319E4284C
:1001A0005F3080000B300D020319E428D33080004B
:1001B00007300D020319E428C63080000F300D020D
:1001C0000319E428D9308000142100088C008C1613
:1001D000EA201E28051006138C1F061705140510AB
:1001E00006130C1F06170514051006138C1E0617A0
:1001F0000514051006130C1E06170514051006132A
:100200008C1D06170514051006130C1D0617051482
:10021000051006138C1C06170514051006130C1C7C
:100220000617051405100800150894001608950017
:100230001708960018089700000898009D301402CF
:10024000031D3429CD301502031D3429DE3016027A
:10025000031D3429D7301702031D342997301802A3
:10026000031D3429051508001B301402031D080066
:10027000DF301502031D08009F301602031D080021
:100280001E301702031D0800D7301802031D080096
:04029000051108004C
:00000001FF
